:020000040000FA
:100000000002040000000000D0100000D01000002A
:10001000D0100000D0100000D0100000D010000060
:10002000D0100000D0100000D0100000D010000050
:10003000D0100000D0100000D0100000D010000040
:10004000D0100000D0100000D0100000D010000030
:10005000D0100000D0100000D0100000D010000020
:10006000D0100000D0100000D0100000D010000010
:10007000D0100000D0100000D0100000D010000000
:10008000D0100000D0100000D0100000D0100000F0
:10009000D0100000D0100000D0100000D0100000E0
:1000A000D0100000D0100000D0100000D0100000D0
:1000B000D0100000D0100000D0100000D0100000C0
:1000C000D0100000D0100000D0100000D0100000B0
:1000D000D0100000D0100000D0100000D0100000A0
:1000E000D0100000D0100000D0100000D010000090
:1000F000D0100000D0100000D0100000D010000080
:10010000D0100000D0100000D0100000D01000006F
:10011000D0100000D0100000D0100000D01000005F
:10012000D0100000D0100000D0100000D01000004F
:10013000D0100000D0100000D0100000D01000003F
:10014000D0100000D0100000D0100000D01000002F
:10015000D0100000D0100000D0100000D01000001F
:10016000D0100000D0100000D0100000D01000000F
:10017000D0100000D0100000D0100000D0100000FF
:10018000D0100000D0100000D0100000D0100000EF
:10019000D0100000D0100000D0100000D0100000DF
:1001A000D0100000D0100000D0100000D0100000CF
:1001B000D0100000D0100000D0100000D0100000BF
:1001C000D0100000D0100000D0100000D0100000AF
:1001D000D0100000D0100000D0100000D01000009F
:1001E000D0100000D0100000D0100000D01000008F
:1001F000D0100000D0100000D0100000D01000007F
:10020000FFFFFF00FFFFFF00D0100000D010000034
:10021000D0100000D0100000D0100000D01000005E
:10022000D0100000D0100000D0100000D01000004E
:10023000D0100000D0100000D0100000D01000003E
:10024000D0100000D0100000D0100000D01000002E
:10025000D0100000D0100000D0100000D01000001E
:10026000D0100000D0100000D0100000D01000000E
:10027000D0100000D0100000D0100000D0100000FE
:10028000D0100000D0100000D0100000D0100000EE
:10029000D0100000D0100000D0100000D0100000DE
:1002A000D0100000D0100000D0100000D0100000CE
:1002B000D0100000D0100000D0100000D0100000BE
:1002C000D0100000D0100000D0100000D0100000AE
:1002D000D0100000D0100000D0100000D01000009E
:1002E000D0100000D0100000D0100000D01000008E
:1002F000D0100000D0100000D0100000D01000007E
:10030000D0100000D0100000D0100000D01000006D
:10031000D0100000D0100000D0100000D01000005D
:10032000D0100000D0100000D0100000D01000004D
:10033000D0100000D0100000D0100000D01000003D
:10034000D0100000D0100000D0100000D01000002D
:10035000D0100000D0100000D0100000D01000001D
:10036000D0100000D0100000D0100000D01000000D
:10037000D0100000D0100000D0100000D0100000FD
:10038000D0100000D0100000D0100000D0100000ED
:10039000D0100000D0100000D0100000D0100000DD
:1003A000D0100000D0100000D0100000D0100000CD
:1003B000D0100000D0100000D0100000D0100000BD
:1003C000D0100000D0100000D0100000D0100000AD
:1003D000D0100000D0100000D0100000D01000009D
:1003E000D0100000D0100000D0100000D01000008D
:1003F000D0100000D0100000D0100000D01000007D
:10040000AF932000007F2200000188000000000060
:100410000C000700200B2100010020001100070044
:10042000000020000000E000020032000000020096
:1004300000000000DA0C0200000000000040DA00BA
:100440000000FE004440A900000020000000E00081
:100450000300320000002000A00188004440A800F2
:100460000000060091018800800078000000EB0089
:1004700015003700E280400032A0B4009101BA00BC
:10048000E280400032A0B4009102BA00E280400055
:1004900032A0B4000002EB00472BDE00F507B200EB
:1004A000602CE10004003A000059EB008301E900F0
:1004B000FDFF3E00040037006128E100010032002A
:1004C0000082EB00040007001101BA000200E00006
:1004D000E8FF3A00000006003159BA008301E90044
:1004E0000C0032002159BA008301E90008003200F3
:1004F0000400E00003003A00E280400032A0B400B3
:10050000F5FF370011D9BA008301E900FAFF3A007C
:100510008100E800E180400032A0B4000000060045
:100520000800FA004047980031079800BE0090008C
:10053000D0112000808F500003003E003E0090004C
:100540000000E00004003A0020002000300798007E
:1005500000CCB3000BE8B700B0C1B300EA06070057
:10056000B0C1B300304798004E409000E606070047
:10057000BE4090004E40900000C068003047980098
:100580003E0090004800DE00204798002E4090007A
:10059000DD060700BE4090002E40900000C06800BD
:1005A000304798003E009000204798002E40900071
:1005B000D5060700BE4090002E40900000C06800A5
:1005C00030479800E0C0B300CF0607003E409000DF
:1005D000E0C0B20030479800000000000000EB00CF
:1005E000000F78000D0037009E007800A0802000EA
:1005F0000080400010407800C30607009E0078008D
:10060000A080200000804000904078003E40900094
:1006100001406800304798001E0FE8009E007800F7
:100620003E009000808F5000EFFF39003E40900068
:10063000B50607000080FA00000006003200FA004C
:10064000881F7800005798006000B80020079800C5
:100650003107980010C0B300504F98000AC8BF007F
:100660000080FB006101B9000080EB008080EB009E
:100670000201400083814800120F9800230F980068
:10068000C0012000010020001E099000AE0990006A
:10069000800F5100818F5900BC043E001E0A90005B
:1006A000AE0A9000046001001C00370034003700DF
:1006B0004F003700B5043700B4043700BC003700E2
:1006C000F4003700B1043700B0043700AF0437003E
:1006D000AE043700AD043700AC043700AB0437007C
:1006E000AA043700F00037004D01370053013700EE
:1006F000790137007A033700750137007603370038
:100700001B04370029043700190437002704370079
:1007100026043700250437004704370010C0B30013
:100720000AE8B7000040EB000BE8B70080C0B30058
:100730000CE8B70010C4B3000DE8B70060C5B30003
:100740000EE8B70020C5B3000FE8B70090C4B300AF
:1007500010E8B70030C5B30011E8B70000C5B3001A
:1007600012E8B700F0C5B30013E8B70020C3B30028
:1007700014E8B700B0002000400798008704370055
:10078000B18020009140780080C9B30080CF500034
:1007900003003A000CC8BF00240507000F00370013
:1007A000B180200091407800E0C9B30080CF5000B4
:1007B00003003A000CC8BF0034E9B7000700370057
:1007C000B180200091407800F0C9B30080CF500084
:1007D00002003A000CC8BF0000E8B700200020006B
:1007E000400798000040EB000BE8B7006B043700AF
:1007F00000C0EB00704F98000BC8BF000080FB00EA
:100800006101B90000F82F00F1FF2F000201400044
:1008100083814800320F9800430F9800F0012000B8
:10082000010020003E099000CE099000800F510089
:10083000818F59004F003E003E0A9000CE0A900082
:10084000046001001F003700210037004900370015
:1008500048003700470037004600370045003700A2
:1008600044003700430037004200370041003700A2
:10087000400037003F0037003E0037003D003700A2
:100880003C00370015003700170037001A0037000A
:10089000380037001B0037001D0037002A003700E2
:1008A0002C0037001D003700320037002C003700C5
:1008B000300037002F0037002C0037001A003700B7
:1008C0001D0037000040EB00704F980029003700F2
:1008D00010C0B300704F98002600370020C0B3004E
:1008E000704F980023003700159320009542780040
:1008F000754F98001F00370032C9BF00704F980035
:100900001C00370020C3B300704F98001900370057
:1009100090C1B300704F980016003700FB04070029
:10092000704F9800130037004193200091407800E9
:10093000714F98000F0037000280200012417800AC
:10094000724F98000B00370020C0B300704F980022
:100950000800370010C0B300704F98000500370042
:10096000C0C8B300704F9800020037000040EB0091
:10097000704F98007E489000E14F400005003A001B
:10098000200020004007980090CCB3000BE8B7008F
:100990000204370030002000400798000040EB00C0
:1009A0000BE8B7007E4890000CE8B700FB03370067
:1009B0000BC8BF000080FB0001002000C800DD0064
:1009C0000000200020408800314088000CC8BF0093
:1009D0000080FB0001002000C001DD0002002000BB
:1009E0002040800031408000000071008180710053
:1009F00020408800314088000DC8BF000080FB0007
:100A0000010020004809DD00C801DE0083017100FB
:100A10004801DD002040800031408000000071006E
:100A20008180710020408800314088000EC8BF00DE
:100A30000081FB0003002000204080003140800046
:100A400000007100818071002040880031408800E2
:100A50000BC8BF000004E00003003D0010C0B3005D
:100A600001E8B700020037000040EB0001E8B700E2
:100A70000CC8BF0003E8B70010C0B30002E8B7001D
:100A800020002000400798000040EB000BE8B70072
:100A9000C2033700200020004007980000CCB300BC
:100AA0000BE8B700BD033700C222A800BB04070053
:100AB0000CC8BF000080FB0051050700200020008B
:100AC0004007980000CCB3000BE8B7000000EB0033
:100AD00010079800E18020009140780000C3B30027
:100AE00080CF50000200360000C3B3000EE8B7000C
:100AF0000FC8BF000004E00043003A0010C0B3007C
:100B00000FE8B7004000370000000000C222A80034
:100B10000DC8BF000080FB00390507001E009000D3
:100B20000000E8001007980012C8BF00C4040700C6
:100B30000FC8BF000080FB003105070013C8BF00CD
:100B4000BF0407000FC8BF000080FB002C05070092
:100B5000C222A90014C8BF00B9040700704F980052
:100B60000FC8BF000080FB002505070015C8BF00A7
:100B7000B3040700604F980011C8BF00E34F500056
:100B800007003A0001812000914078007E489000E3
:100B900080CF500002003A000040EB000BE8B700A5
:100BA00011C8BF00E34F5000070032000181200050
:100BB000914078006E48900080CF500002003A00CB
:100BC0000040EB000BE8B70011C8BF000004E000D4
:100BD00002003A000040EB000BE8B7000BC8BF0072
:100BE0000004E00005003A00C222A8000EC8BF00C1
:100BF0000080FB001007980003003700480407003E
:100C000040012000FE0407000EC8BF008080FB00EA
:100C10001E009000808F5000BBFF3E005F03370036
:100C2000BA040700C222A900200020004007980053
:100C30000040EB000BE8B700580337000DC8BF00B9
:100C40007F0407000EC8BF007D0407000FC8BF0067
:100C50007B04070010C8BF00790407000CC8BF0060
:100C60000004E00004003A000BC8BF000080FB0055
:100C7000E30407001100370060C9B300404F98003B
:100C8000030037004E4890000040E900404F9800B4
:100C90000000200001002F00870407000080FB00F7
:100CA000610060000004A2000004E00003003A00BC
:100CB0004E4890000004E000F2FF3A0020002000BF
:100CC000400798000040EB000BE8B7003303370003
:100CD0000040EB00504F98006000B80020079800DB
:100CE0003107980060C9B300404F98000EC8BF009C
:100CF000E34F500002003E0040C0B3000EE8B700D2
:100D0000E18020009140780000C2B30080CF500005
:100D10000200360000C2B3000EE8B7002040800099
:100D200031408000404088000BC8BF000080FB00BD
:100D30004800DD00000F78000CC8BF000080FB00F9
:100D40001E0F7000801120009E0F1000050036005D
:100D5000200020004007980000CCB3000BE8B7004B
:100D60000E03370000000000D18020009140780081
:100D7000614F98000040EB00204F98000DC8BF0065
:100D80000080FB000000A200610060000004E000A1
:100D9000B20032000000EB0010079800AB003700F3
:100DA0005E4890000004E000090032001E00900040
:100DB000610060000004A2000004E00004003A00AA
:100DC0000FC8BF000034A0001D0407000200370058
:100DD0000FC8BF001A040700204080003140800087
:100DE0002B0407001E009000EA004000A0802000B5
:100DF000008040001040780011040700228120008C
:100E0000124178001E009000EA004000A0802000FF
:100E10000080400010407800804F510021003200D7
:100E20002040800031408000F2FF2F0003002000AE
:100E300000027800810278000200780083007800C8
:100E400000016200018062006102B800540F980046
:100E5000650F98005E089000EE089000C000DD006D
:100E600000002000500F9800610F98005E0890006D
:100E7000EE0890006112B800540F9800650F9800BA
:100E80005E099000EE0990000200700083807000FF
:100E900020079800310798006E4890000DE8B700D1
:100EA0000200370020C0B3000DE8B70000000000CA
:100EB0005E4890000004E00002003A00200020009C
:100EC0004F0407000DC8BF000080FB004200DE0099
:100ED000610060000004E000250032002181200054
:100EE00091407800714F980060C9B300404F98005E
:100EF000160037005E4890000004E0000900320050
:100F00001E009000610060000004A2000004E000E8
:100F100004003A0011C8BF000034A000C803070055
:100F20000200370011C8BF00C50307002E00900063
:100F3000D70307000040EB00C1030700704F980083
:100F40004E4890000040E900404F98002181200069
:100F5000914078007E48900080CF50001F003A00FA
:100F60004E4890000004E000E2FF3A001B0037000A
:100F70000DC8BF000080FB004300DE006100600080
:100F80000004E0001200320060C9B300404F980036
:100F9000030037004E4890000040E900404F9800A1
:100FA0000000200001002F00C30307000080FB00A9
:100FB000610060000004A2000004E00007003A00A5
:100FC0004E4890000004E000F2FF3A0003003700B2
:100FD0000EC8BF000080FB00090407005E489000B7
:100FE0000004E0000B0032001E0090006100600071
:100FF0000004E0000D0032002040800031408000FD
:1010000061004000E08048002040880031408800B6
:101010000600370020408000314080006100400021
:10102000E080480020408800314088004E48900011
:101030000004E00002003A0000C8B300204F98000E
:101040001E0090000000E800100798001E009000AD
:101050009E0F500052FF39001A0137000000EB00CC
:1010600010079800B00037000000000001C8BF0062
:101070000004E0002C00320020408000314080005D
:10108000F2FF2F00030020000002780081027800A8
:101090000200780083007800000162000180620095
:1010A0006102B800740F9800051798007E08900040
:1010B0008E109000C000DD0000002000700F98002E
:1010C000011798007E0890008E1090006112B80001
:1010D000740F9800051798007E0990008E119000FB
:1010E0000200700083807000E00F5000E08F580015
:1010F0000300320002C8BF000004E0000A00320012
:10110000D0C4B3004E0307000040EB004C030700BF
:1011100003C8BF004A0307000040EB004803070074
:101120000040EB0002E8B7005E4890000004E000D9
:10113000090032001E009000610060000004A2005F
:101140000004E00004003A000FC8BF000034A00013
:101150003B030700020037000FC8BF003803070039
:101160002040800031408000490307001E009000AD
:10117000EA004000A080200000804000104078007D
:101180002F03070022812000124178001E009000EA
:10119000EA004000A080200000804000104078005D
:1011A000804F51001F0032002040800031408000FD
:1011B000F2FF2F0003002000000278008102780077
:1011C0000200780083007800000162000180620064
:1011D0006102B80014179800251798001E1090009F
:1011E000AE109000C000DD00000020001017980035
:1011F000211798001E109000AE1090006112B800E8
:1012000014179800251798001E119000AE11900039
:10121000020070008380700020079800310798005A
:10122000060037000DC8BF008040780000C8B3003A
:1012300000C060000044A0000DE8B7005E489000C8
:101240000004E0002F0032001E00900061006000EA
:101250000004E00031003200204080003140800076
:1012600061004000E0804800204088003140880054
:101270002040800031408000F2FF2F00030020005A
:101280000002780081027800020078008300780074
:1012900000016200018062006102B800341798000A
:1012A000451798003E109000CE109000C000DD0061
:1012B0000000200030179800411798003E10900061
:1012C000CE1090006112B8003417980045179800AE
:1012D0003E119000CE1190000200700083807000DB
:1012E000F2FF2F0003002000820F5000838F580070
:1012F0000A003A0003C8BF000040E80003E8B70056
:10130000060037002040800031408000610040002E
:10131000E080480020408800314088001E00900096
:101320000000E800100798001E0090009E0F50007B
:101330004DFF3900000000000DC8BF000004E000B0
:1013400060003D0010C8BF00BD02070040408000A3
:10135000CF0207000040EB00B90207005E48900092
:101360000004E00002003A001000200024030700FF
:1013700060C9B300404F98000DC8BF000080FB005B
:101380004500DE00610060000004A2000004E000EF
:101390002E003A002E009000BE009000E00F50009A
:1013A000E08F58002900320023812000934178000B
:1013B000734F9800170037002E009000BE00900079
:1013C000610160006000B8000300200002007000AE
:1013D000838070000000E0000400320011C8BF00EC
:1013E0000034A000960207000200370011C8BF00B9
:1013F000930207002E009000A50207000040EB00BA
:101400008F020700704F98004E4890000040E9009E
:10141000404F980021812000914078007E48900044
:1014200080CF500003003A004E4890000004E000D6
:10143000E1FF3A004E4890000004E00021003A002D
:1014400000C8B300204F98001E0037000DC8BF0031
:101450000080FB004600DE00610060000004E00048
:1014600015003200030037004E4890000040E900AC
:10147000404F98000000200001002F008E0207005E
:101480000080FB00610060000004A2000004E00096
:1014900003003A004E4890000004E000F2FF3A00DA
:1014A0004E4890000004E00006003A0010C8B30067
:1014B000204F9800030037000EC8BF000080FB00DB
:1014C000CF02070020002000400798002E4890001F
:1014D0000BE8B700310137000040EB00504F980097
:1014E0000BC8BF000080FB004800DD00000F780043
:1014F0000CC8BF000080FB001E0F7000D1802000D0
:1015000091407800714F9800801120009E0F1000CC
:101510000200360080112000000F78000000EB0070
:1015200010079800840037000000000001C8BF00C9
:101530000004E0002C003200204080003140800098
:10154000F2FF2F00030020000002780081027800E3
:1015500002007800830078000001620001806200D0
:101560006102B80054179800651798005E1090004B
:10157000EE109000C000DD00000020005017980021
:10158000611798005E109000EE1090006112B80094
:1015900054179800651798005E119000EE119000A6
:1015A0000200700083807000E00F5000E08F580050
:1015B0000300320002C8BF000004E0000A0032004D
:1015C000D0C4B3001E0207000040EB001C0207005D
:1015D00003C8BF001A0207000040EB001802070012
:1015E0000040EB0002E8B7005E4890000004E00015
:1015F000090032001E009000610060000004A2009B
:101600000004E00004003A007E4890000034A0008E
:101610000B020700020037007E4890000802070016
:101620002040800031408000190207001E00900019
:101630000084E8000040EB000102070080407800D1
:10164000A080200000004400014878005E4890001F
:101650000004E0002F0032001E00900061006000D6
:101660000004E00031003200204080003140800062
:1016700061004000E0804800204088003140880040
:101680002040800031408000F2FF2F000300200046
:101690000002780081027800020078008300780060
:1016A00000016200018062006102B80074179800B6
:1016B000051F98007E1090008E189000C000DD007D
:1016C0000000200070179800011F98007E10900005
:1016D0008E1890006112B80074179800051F9800CA
:1016E0007E1190008E1990000200700083807000BF
:1016F000F2FF2F0003002000820F5000838F58005C
:101700000A003A0003C8BF000040E80003E8B70041
:10171000060037002040800031408000610040001A
:10172000E080480020408800314088001E00900082
:101730000000E800100798001E0090009E0F500067
:1017400079FF39009E0178006380410040079800CE
:101750000040EB000BE8B7009E80E800A08020006E
:10176000808040000040EB00804878008B0037000C
:101770000BC8BF00B20107000CC8BF00B0010700D2
:101780000DC8BF00AE0107000EC8BF00AC010700C6
:1017900030002000400798000040EB000BE8B70045
:1017A0000040EB000CE8B7007C0037000040EB0085
:1017B000404F9800160037004E4890000080FB0014
:1017C0008080E800A0802000008040001040780069
:1017D0009B010700704F98000BC8BF008080FB0082
:1017E0004E4890000080FB000000E800808F500011
:1017F00002003A007E4890000CE8B700500020003C
:10180000FF0107004E4890000040E800404F98005C
:101810004E489000E34F5000E7FF360040002000A4
:10182000400798000040EB000BE8B7000040EB00D9
:101830000DE8B70059003700C180200091407800C2
:10184000714F9800D280200012417800624F9800BA
:101850000040EB00304F98000040EB00404F9800F4
:101860000040EB00304F9800260037005000200069
:10187000E3010700BE4890006E48900080CF500002
:1018800016003900CE4890007E48900080CF50006E
:10189000120031004E4890000080FB000084E800F8
:1018A0003E4890000080FB00E4004000A080200043
:1018B00000804000104078006101070080407800FF
:1018C000A080200000004400014878004E489000AD
:1018D0000040E800404F9800070037003E48900065
:1018E0000080FB00E4004000A08020000080400059
:1018F00010407800520107003E4890000040E80088
:10190000304F9800B1802000914078003E48900010
:1019100080CF5000D5FF3E000A0037004E489000AF
:101920000080FB008080E800A080200080804000D4
:101930000040EB00804878004E4890000040E800EE
:10194000404F9800CE4890007E48900080CF5000D5
:10195000F2FF39004E4890000080FB006300400019
:10196000400798000040EB000BE8B7004E4890009D
:101970000080FB008080E800A08020008080400084
:101980000040EB0080487800040037002000200071
:101990004007980090CCB3000BE8B700CE00900051
:1019A0000E509000DEFA07004F0478000080FA0025
:1019B000000006000A00FA000040EB0070479800A3
:1019C0000040EB00504798000040EB004047980073
:1019D0000000EB00100798000000EB00000F7800FB
:1019E00067010700D2010700C022A900C222A90096
:1019F0000040EB0060479800A0C0B30032E9B70098
:101A000020C0B30031E9B700000037006E409000FD
:101A10000004E00003003A00B2010700004F980004
:101A200002003700AF010700004F98006E409000A1
:101A30000004E00008003A000E489000FB4F500000
:101A400005003A0010C0B300604798000E489000AF
:101A500050479800EDFF37006E409000E14F500076
:101A600009003A008E48900041479800DE409000FF
:101A70000E48900000C068005047980020C0B30096
:101A800060479800E1FF37006E409000E24F500041
:101A90000B003A00DE4090000E48900000C0680045
:101AA000504798000E4890000080FB004800DD0081
:101AB0001007980030C0B30060479800D3FF37008C
:101AC0006E409000E34F50000C003A00DE40900062
:101AD0000E48900000C06800504798000E489000E3
:101AE0008080FB001E00900001007000100798002D
:101AF00040C0B30060479800C4FF37006E409000BC
:101B0000E44F50000F003A00DE4090000E48900075
:101B100000C06800504798000E489000EE4F5000FB
:101B200005003A0050C0B300604798000000EB0089
:101B3000000F7800B5FF37000040EB0060479800C9
:101B4000B2FF37006E409000E54F500017003A009A
:101B50001E0090009E0F100014003D007011200028
:101B60009E0F100011003C00DE4090000E489000D7
:101B700000C06800504798009E007800A0802000B8
:101B8000008040008E489000014878001E0FE80059
:101B9000000000001E0090009E0F10009BFF3A0006
:101BA00060C0B3006047980098FF37006E40900017
:101BB000E64F500012003A008E4890005E409000C0
:101BC00080CF500007003A001E0090000000E000A7
:101BD00004003400000000004E40900097FA070017
:101BE0000700370000CBB3000AE8B70010CCB30001
:101BF0000BE8B700210020004E40900048FA070093
:101C00000040EB00604798000000EB0010079800D0
:101C10000040EB00404798000040EB007047980000
:101C20000000EB00000F780078FF37000200FA0098
:101C3000004F780041E2A9000040EB0038E9B7000E
:101C400030C0B3009E4F10000700360010C0B30034
:101C500038E9B700C0C0B30036E9B7000000EB00B8
:101C6000101288001E00370020C0B3009E4F1000E5
:101C70000500360030C0B30036E9B7000000EB00C5
:101C8000101288001600370010C0B3009E4F1000DD
:101C90000500360020C0B30036E9B7008000200000
:101CA000101288000E00370010C0B3009E4F1000C5
:101CB00005003A0010C0B30036E9B700C0012000AB
:101CC00010128800060037001E04E00004003A00ED
:101CD0000040EB0036E9B700D00120001012880068
:101CE00042A2A8004302A8000000EB0020128800D6
:101CF0000000EB000012880041E2A80036C9BF00D6
:101D00000080FB000080FA00000006000000FA00DE
:101D100036C9BF000080FB000080FA00000006000A
:101D20000000FA00816C20009140780000CEB300E2
:101D300000C06000C8E6B700CB02A90040C6B300EF
:101D4000C8000700CB02A80040C6B300C5000700CA
:101D5000CB02A900816C20009140780000CEB30036
:101D600000C060000034A000C8E6B700000000001A
:101D70000080FA00000006000000FA00CAC2A800B5
:101D800040C6B300B7000700CAC2A9004001200046
:101D90009B0007000080FA00000006000000FA0027
:101DA000CAC2A800C8C2A90041E2A900CEE2A900A7
:101DB000CF02A900CEC2A900816A2000914078001C
:101DC00000CEB30000C060007040B300A8E6B700CA
:101DD000916C20009140780000CEB30000C06000FC
:101DE0007040B300C9E6B700816C200091407800D4
:101DF00000CEB30000C060000034A000C8E6B70009
:101E0000C902A900C8E2A800C922A900CB02A90002
:101E1000CAE2A900CB22A9004001200078000700F7
:101E200036C9BF0081FF0700CAC2A90040012000D7
:101E300073000700D0FF07000080FA0000000600D2
:101E40000400FA002047980000C8B300104798002B
:101E50000040EB00004F78002E4090000080FB0017
:101E60004012880085C0BF00644060000004E000AC
:101E7000FCFF320040128000204798008540A900F6
:101E80002E4090000080FB000080FA000000060059
:101E90000200FA00000F78001E0078004800DE0003
:101EA000E7FF07001E007800E5FF07000080FB0049
:101EB0000080FA00000006000400FA00008FBE0057
:101EC0001E00BE004808DE0001002000DCFF070005
:101ED0001E00BE004008DE0001002000D8FF070001
:101EE0001E00BE004809DD004800DE000000710051
:101EF000C808DE00D2FF07001E007800D0FF0700F0
:101F00000080FB000080FA00000006000000FA00DC
:101F1000CAC2A80041E2A900A8C6BF00F041B300B0
:101F2000A8E6B700916C20009140780000CEB30085
:101F300000C06000C9E6B700816C200091407800C5
:101F400000CEB30000C06000C8E6B700CEE2A90032
:101F5000CF02A900CEC2A900C922A800CB22A900A5
:101F6000C902A800CB02A900C8E2A800CAE2A900E1
:101F7000C8C2A800CAC2A9000080FA00000006007A
:101F80000000FA004507A9000080EB0060198800F6
:101F90004227A900C022A90041168000007C200031
:101FA000008070004016880061168000F0FB2F0052
:101FB0000080600060168800CB62A900C962A90099
:101FC000C002A900C202A800416A20009140780026
:101FD00000CEB30000C060005040B300A4E6B700DC
:101FE000416C20009140780000CEB30000C060003A
:101FF0003040B300C4E6B7000080FA0000000600DD
:102000000600FA00200798000000EB001007980077
:102010000E0037000040EB00004F7800050037004D
:10202000A0CFB3000F0007001E4078000040E8007A
:10203000004F78001E407800E34F5000F8FF360054
:102040001E0090000000E800100798009E0090001D
:102050002E009000808F5000EEFF39000080FA00C3
:10206000000006000400FA00204798000040EB0042
:10207000004F78000F003700000000000000000053
:102080000000000000000000000000000000000050
:102090000000000000000000000000000000000040
:1020A00000000000000000001E4078000040E80032
:1020B000004F78009E4078002E40900080CF500066
:1020C000EDFF39000080FA00000006000000FA0071
:1020D00022C2BF00614060000080FB000080FA0067
:1020E000000006000000FA0022C2BF00614060004C
:1020F0000004E000FCFF3200301180000080FB0093
:102100000080FA00000006000200FA00004F78008C
:1021100023C2BF00624060000004E000FCFF3A0000
:102120001E00FB00201188000080FA00000006005D
:102130000000FA0020022000401188000000EB009F
:10214000001188002062A8000000EB001011880038
:1021500021E2A8002342A8008560A9000080FA00BF
:102160000000060034090000020000000200000028
:102170000100000000080000340100000000000021
:10218000360900000200000002000000010000000B
:1021900038090000020000000000000000000000FC
:1021A0000000FE00FFFFFF00FFFFFF00FFFFFF003A
:1021B000FFFFFF00FFFFFF00FFFFFF00FFFFFF002B
:1021C000FFFFFF00FFFFFF00FFFFFF00FFFFFF001B
:1021D000FFFFFF00FFFFFF00FFFFFF00FFFFFF000B
:1021E000FFFFFF00FFFFFF00FFFFFF00FFFFFF00FB
:020000040001F9
:00000001FF
